:0400000071EF22F08A
:1000080000C016F001C015F0E1CF17F0E2CF18F0EC
:100018009DAA5BD09EAA59D0AECFFEF0ABA20FD05E
:10002800AB98AECFFEF0AB88010E01011525006E2E
:10003800000E1621016E00C015F101C016F1ABA427
:100048000FD00101AB9EAB8E010E1525006E000E80
:100058001621016E00C015F101C016F1AECFFEF0F9
:100068000001FE510D0A07E0F751000802E1F651C0
:100078004E0801E313D0010EF86F000EF96FA40EBD
:10008800F625E16E000EF721E26EE66AF6C0F4F09E
:10009800F7C0F5F0F66BF76BFE6B16D0A40EF625DD
:1000A800E16E000EF721E26EFEC0E6FFF6C0F4F046
:1000B800F7C0F5F0010EF625006E000EF721016E6F
:1000C80000C0F6F001C0F7F09E9A9DA01FD09EA038
:1000D8001DD00001010EFA25006E000EFB21016EF5
:1000E80000C0FAF001C0FBF0000EFB5D02E1080E53
:1000F800FA5D07E3FA6BFB6B010EFC6F000EFD6FF8
:100108009D900B0ECF6EDB0ECE6E9E9016C000F04B
:0E01180015C001F017C0E1FF18C0E2FF110092
:0E012600026A016A006A086A036A000E12008B
:0E013400ACB202D00000FCD75DC1ADFF1200DE
:0C01420072B201D0FDD75DC173FF120046
:10014E000B820BAEB1EF00F0036802680168006825
:08015E000A360232FF0E120006
:100166000B840BAEBEEF00F0010E036E026A016A4D
:0A017600006A0A360232FF0E120082
:080180000AAE029E000E1200FF
:100188000CB006EF01F00CA2ACEF01F00E6A000E05
:1001980002641DEF01F0F00E0214D8A4E8EF00F09D
:1001A800023A01380F0B02260138F00B016E0038B5
:1001B8000F0B01260038F00B006E08380F0B0026D5
:1001C8000838F00B086E0E84D89002BE01EF01F0DB
:1001D80008360036013602360E2A02BE01EF01F05B
:1001E80008360036013602360E2A02BE01EF01F04B
:1001F80008360036013602360E2A0E500364A2EF86
:1002080001F0035E0BBC08AEA7EF01F0D880800EAA
:1002180008640030000E002201220222D8A0A7EFB5
:1002280001F0023201320032034AACEF01F0A7EFCD
:1002380001F001C002F000C001F008C000F0086A37
:10024800000E0E86026454EF01F0F00E0214D8A4DA
:100258003CEF01F0023A01380F0B02260138F00B8F
:10026800016E00380F0B01260038F00B006E0E846B
:10027800D89002BE01EF01F00036013602360E2A90
:1002880002BE01EF01F00036013602360E2A02BE28
:1002980001EF01F00036013602360E2A01EF01F0B7
:1002A80001C002F000C001F0006A000E0E960E8830
:1002B800026481EF01F0F00E0214D8A46CEF01F093
:1002C800023A01380F0B02260138F00B016E0E843A
:1002D800D89002BE01EF01F0013602360E2A02BEA6
:1002E80001EF01F0013602360E2A02BE01EF01F0DD
:1002F800013602360E2A01EF01F001C002F0016A50
:10030800000E0E860264B1EF01F0F00E0214D8A4BC
:1003180090EF01F0023A0E84D89002BE01EF01F08E
:1003280002360E2A02BE01EF01F002360E2A02BE84
:1003380001EF01F002360E2A01EF01F0010E0C6EFA
:100348000EDFB4EF01F0020E0C6E16DFB4EF01F011
:10035800040E0C6EF8DEB4EF01F0080E0C6EDFDE52
:02036800120081
:10036A00F250026EF29E0500FF6A0150FE6E0050C6
:08037A00FD6E02BEF28E1200BE
:10038200C7B409D01F0EC514016E0150000A03E163
:0A039200010E006E01D0006A120097
:10039C00086A080E0C6E003408360450085ED8B09B
:0E03AC0002D00826D89000360C2EF5D712008D
:0803BA000B6A0B86FF0E120016
:1003C2000D6A086A0050D8B4000C04180A6E0ABEFE
:1003D2000D1E0B6A04AE02D0041E042A00AE02D027
:1003E200001E002A005004100A6E0ABE1FD00450DC
:1003F200085E003600340836045008260036060E21
:100402000C6E00340836045000B0085E00A00826C6
:1004120000360C2EF6D700A008260BB015D00DAE74
:10042200000C001E002A081E082A000C04AE09D087
:1004320000BE04D00050086E006AF1D7006A002A9C
:10044200000C001E0B2AD3D7082A0450085CD8A43B
:0E045200E6D7086A002A00AEE2D7FF0C1200BF
:10046000086A096A000E07620364B5EF02F00250E1
:1004700006180A6E075003267E0ED8A046EF02F03B
:10048000035ED8B0B9EF02F04AEF02F0035ED8A0E5
:10049000BDEF02F0028E068E02C00EF001C00BF01E
:1004A00000C00DF000500402F4CF0CF00150050222
:1004B000F4CF00F0F3CF08F00402F3500C26F45010
:1004C0000822000E00220D500502F3500C26F450B5
:1004D0000822000E002202500402F3500826F450B5
:1004E000002202500502016A000E0122F35000268C
:1004F000F45001220D500602F3500826F450002259
:10050000026A000E012202220B500602F35000265E
:10051000F4500122000E02220E500602F350012672
:10052000F450022202BE9DEF02F00836003601367A
:1005300002360306D8B4BDEF02F0B0EF02F0D88067
:10054000800E08640030000E002201220222D8A092
:10055000B0EF02F0023201320032034AB9EF02F08A
:100560000AAE029E000EBFEF02F0010EDCDDBFEF0F
:1005700002F0020EECDDBFEF02F0040EF4DD12001B
:100580000B800BAECCEF02F0026A0AAEFF0E026ED9
:0C059000016E006E0A360232FF0E1200EF
:10059C00025006180E6E086A096A0B6A035007644B
:1005AC00C1EF03F006500A6E068E028E03500B6EDE
:1005BC000750036E000E0B6411EF03F00B50075E37
:1005CC00D8B4B2EF03F0070E076480EF03F0075EB8
:1005DC0000C008F001C000F002C001F0026A074E32
:1005EC00B2EF03F0076455EF03F0075E00C008F0AC
:1005FC0001C000F0016A074EB2EF03F0076433EF5D
:10060C0003F0075E00C008F0006A074EB2EF03F07B
:10061C0007641AEF03F00AC002F005C001F004C031
:10062C0000F0086ADEEF04F0030E076425EF03F018
:10063C00075E08380F0B086E074EB2EF03F0D89028
:10064C000832074EB2EF03F0D8900832074EB2EFE3
:10065C0003F0D8900832B2EF03F0030E076444EFB6
:10066C0003F0075E08380F0B086E0038F00B0826F5
:10067C0000380F0B006E074EB2EF03F0D89000322B
:10068C000832074EB2EF03F0D89000320832074E12
:10069C00B2EF03F0D89000320832B2EF03F0030E41
:1006AC0007646CEF03F0075E08380F0B086E003818
:1006BC00F00B082600380F0B006E0138F00B0026EB
:1006CC0001380F0B016E074EB2EF03F0D8900132D8
:1006DC0000320832074EB2EF03F0D89001320032EC
:1006EC000832074EB2EF03F0D890013200320832D4
:1006FC00B2EF03F0030E07649DEF03F0075E0838BA
:10070C000F0B086E0038F00B082600380F0B006E2C
:10071C000138F00B002601380F0B016E0238F00B7C
:10072C00012602380F0B026E074EB2EF03F0D89081
:10073C000232013200320832074EB2EF03F0D89089
:10074C000232013200320832074EB2EF03F0D89079
:10075C000232013200320832096A000E0EAEA6EFE8
:10076C0004F0081E001E011E021E082A002201228F
:10077C000222A6EF04F00750D8A4C7EF03F0DEEF77
:10078C0004F0096A02C00AF0028E068E0750035C60
:10079C00076ED8B499EF04F0070E076467EF04F006
:1007AC00075E0450096E0550046E0650056E066A0D
:1007BC00074E99EF04F0070E07643CEF04F0075E58
:1007CC000450096E0550046E056A074E99EF04F04B
:1007DC00070E07641AEF04F0075E0450096E046AF2
:1007EC00074E99EF04F0070E076401EF04F00AC0FE
:1007FC0002F0DEEF04F0030E07640CEF04F0075E6A
:10080C0009380F0B096E074E99EF04F0D890093296
:10081C00074E99EF04F0D8900932074E99EF04F087
:10082C00D890093299EF04F0030E07642BEF04F013
:10083C00075E09380F0B096E0438F00B09260438D3
:10084C000F0B046E074E99EF04F0D8900432093266
:10085C00074E99EF04F0D89004320932074E99EF05
:10086C0004F0D8900432093299EF04F0030E0764B7
:10087C0053EF04F0075E09380F0B096E0438F00BC8
:10088C00092604380F0B046E0538F00B04260538C6
:10089C000F0B056E074E99EF04F0D8900532043219
:1008AC000932074E99EF04F0D89005320432093220
:1008BC00074E99EF04F0D89005320432093299EFC3
:1008CC0004F0030E076484EF04F0075E09380F0B85
:1008DC00096E0438F00B092604380F0B046E05382A
:1008EC00F00B042605380F0B056E0638F00B0526A9
:1008FC0006380F0B066E074E99EF04F0D8900632AF
:10090C00053204320932074E99EF04F0D8900632C2
:10091C00053204320932074E99EF04F0D8900632B2
:10092C00053204320932086A000E0EAEA6EF04F04E
:10093C00091E041E051E061E092A04220522062273
:10094C0009500826045000220550012206500222AC
:10095C000EBEBDEF04F0D8A0CCEF04F00232013291
:10096C0000320832033ECCEF04F0D8EF04F0D8B0DC
:10097C00D2EF04F0000E081E001E011E021E082AF3
:10098C000022012202220A7ED2EF04F0010E0C6E2C
:10099C00C4EC00F0E0EF04F0020E0C6EC4EC00F0BE
:1009AC00E0EF04F0040E0C6EA7EC00F0E0EF04F0A6
:0609BC00000E0C6E12009B
:1009C2009E9657C1C9FF20C058F121C059F122C0DB
:1009D2005AF123C05BF1C7A421D02050211022106C
:1009E20023101BE00101585159115A115B110EE1FC
:1009F20030C0E1FF31C0E2FF040EE66E2EC000F00F
:100A02002FC001F0B1DC010E006E3AD0010E0101DF
:100A1200585F000E595B5A5B5B5BDDD720C058F113
:100A220021C059F122C05AF123C05BF19EB621D0F8
:100A320020502110221023101BE00101585159119E
:100A42005A115B110EE130C0E1FF31C0E2FF040E2A
:100A5200E66E2EC000F02FC001F086DC010E006EA3
:100A62000FD0010E0101585F000E595B5A5B5B5BB0
:100A7200DDD7C5BC02D0006A03D0C584020E006E69
:020A8200120060
:040A8400C584120013
:100A88000134083609360450085E0550D8A0053CE4
:100A9800095E003601360F0E0C6E01340836093631
:100AA800045000A006D0085E0550D8A0053C095E99
:100AB80005D008260550D8B0053C09260036013671
:100AC8000C2EEBD700B006D0045008260550D8B03D
:080AD800053C09260000120094
:100AE00020C059F121C05AF122C05BF123C05CF152
:100AF0000101576B586B5851120802E157518E088B
:100B000008E33FDC005201E004D00101574B582BB1
:100B1000F2D70101120E585D02E18F0E575D03E31B
:100B20007B0E006E24D0C580C5A020D0205021109F
:100B3000221023101AE059515A115B115C110EE179
:100B400030C0E1FF31C0E2FF050EE66E2EC000F0BE
:100B50002FC001F00ADC010E006E09D0010E010168
:100B6000595F000E5A5B5B5B5C5BDED7006A12006C
:100B70000B6A0C6A086A0350D8B43CEF06F002C056
:100B80000AF0028E9E0E035E03AE2CEF06F0036C9D
:100B9000080E035CD8A0F9EF05F0036E083600C01C
:100BA00008F001C000F002C001F0026A080E035C08
:100BB000D8A0F9EF05F0036E083600C008F001C0B8
:100BC00000F0016A080E035CD8A0F9EF05F0036E8F
:100BD000083600C008F0006A080E035CD8A0F9EFE0
:100BE00005F0036E0836086A0350D8A4D89005EFC4
:100BF00006F00350D8B405EF06F0D8900232013267
:100C000000320832032EFDEF05F00BBC08A016EFF2
:100C100006F0D8A016EF06F0082AD8B4002AD8B4F7
:100C2000012AD8B4022A02BE40EF06F00AAE3CEF19
:100C300006F0021E011E001E081E082AD8B4002A53
:100C4000D8B4012AD8B4022A3CEF06F0026A016A3D
:100C5000006A086A3CEF06F00B800BAE46EF06F028
:100C6000026A0AAE46EF06F0026E016E006E086E72
:100C70000A36023246EF06F00C6A000E47EF06F025
:100C8000010E0C6E000E7CDC47EF06F0FF0E0250EA
:100C9000036E0150026E0050016E0850006E12008B
:100CA0001FDF3DC057F18DDE00C054F10050FF0A38
:100CB000D8B4C69E53C157F184DE00C054F1E2DEC1
:060CC00054C100F0120017
:060CC600067E69DC12004D
:100CCC006E0E0101525DD8A0CAD0640E046E52C1E2
:100CDC0000F0CEEC01F0120E0024056E066A000E38
:100CEC00062205C000F006C001F0000E06BEFF0E85
:100CFC00026E036E00360090013602360336003663
:100D0C0000900136023603362F0E0024F66E490E83
:100D1C000120F76E000E0220F86E0900F5CF00F0EE
:100D2C000900F5CF01F00900F5CF02F00900F5CF6D
:100D3C0003F0000E046E000E056E000E066E7E0EA5
:100D4C00076E30EC02F000C053F101C054F102C048
:100D5C0055F103C056F1640E046E52C100F0CEEC96
:100D6C0001F008C000F00A0E046ECEEC01F0090E82
:100D7C000024056E066A000E062205C000F006C0AF
:100D8C0001F0000E06BEFF0E026E036E00360090E0
:100D9C000136023603360036009001360236033631
:100DAC002F0E0024F66E490E0120F76E000E022065
:100DBC00F86E0900F5CF00F00900F5CF01F009003D
:100DCC00F5CF02F00900F5CF03F053C104F054C184
:100DDC0005F055C106F056C107F030EC02F000C02A
:100DEC0053F101C054F102C055F103C056F10A0E83
:100DFC00046E52C100F0CEEC01F008C000F000C04F
:100E0C0001F0000E026E036E046E01360190023684
:100E1C0003360436013601900236033604362F0EA3
:100E2C000124F66E490E0220F76E000E0320F86EB8
:100E3C000900F5CF00F00900F5CF01F00900F5CF5E
:100E4C0002F00900F5CF03F053C104F054C105F0D2
:100E5C0055C106F056C107F030EC02F0B1D052513A
:100E6C000A08D8B07ED00A0E046E52C100F0CEEC47
:100E7C0001F0090E0024056E066A000E062205C05C
:100E8C0000F006C001F0000E06BEFF0E026E036EEF
:100E9C0000360090013602360336003600900136DB
:100EAC00023603362F0E0024F66E490E0120F76E23
:100EBC00000E0220F86E0900F5CF00F00900F5CF06
:100ECC0001F00900F5CF02F00900F5CF03F0000E98
:100EDC00046E000E056E000E066E7E0E076E30EC74
:100EEC0002F000C053F101C054F102C055F103C02F
:100EFC0056F10A0E046E52C100F0CEEC01F008C09F
:100F0C0000F000C001F0000E026E036E046E01369C
:100F1C000190023603360436013601900236033650
:100F2C0004362F0E0124F66E490E0220F76E000EC9
:100F3C000320F86E0900F5CF00F00900F5CF01F0A1
:100F4C000900F5CF02F00900F5CF03F053C104F00E
:100F5C0054C105F055C106F056C107F030EC02F053
:100F6C002FD052C100F0000E016E026E036E0036DF
:100F7C0000900136023603360036009001360236F8
:100F8C0003362F0E0024F66E490E0120F76E000E6C
:100F9C000220F86E0900F5CF00F00900F5CF01F042
:100FAC000900F5CF02F00900F5CF03F0000E046E36
:100FBC00000E056E000E066E7E0E076E30EC02F013
:020FCC00120011
:100FCE000B6A0C6A0A6A086A0350D8B46FEF08F00D
:100FDE00028E9E0E035E03BEFAEF07F0D8B4FAEF50
:100FEE0007F05FEF08F0036C080E035CD8A02CEF3F
:100FFE0008F0036E083600C008F001C000F002C011
:10100E0001F0026A080E035CD8A02CEF08F0036E04
:10101E00083600C008F001C000F0016A080E035C3B
:10102E00D8A02CEF08F0036E083600C008F0006A56
:10103E00080E035CD8A02CEF08F0036E0836086A81
:10104E000350D8A4D89038EF08F00350D8B438EF36
:10105E0008F0D8900232013200320832032E30EFFF
:10106E0008F00BBC08A049EF08F0D8A049EF08F033
:10107E00082AD8B4002AD8B4012AD8B4022A02BE4B
:10108E0073EF08F00AAE6FEF08F0021E011E001E8D
:10109E00081E082AD8B4002AD8B4012AD8B4022AC5
:1010AE006FEF08F0026A016A006A086A6FEF08F0D3
:1010BE000B800BAE79EF08F0026A0AAE79EF08F0FA
:1010CE00026E016E006E086E0A36023279EF08F07B
:1010DE00000E0C6A7AEF08F0010E0C6EC0EC02F0F6
:1010EE007AEF08F0FF0E0250036E0150026E0050B0
:0810FE00016E0850006E1200A3
:1011060003500718D8A497EF08F002500618D8A481
:1011160097EF08F001500518D8A497EF08F0005093
:0E1126000418D8B4D8841200D8941200120015
:101134000B6A0A6A096A086A0E6A0334083604509C
:10114400085E0550D8A0053C095E0650D8A0063CB0
:101154000A5E0750D8A0073C0B5EE86AD8A0010ECF
:101164000E5E0336070E0C6E0334083609360A3653
:101174000B360E36045003A012D0085E0550D8A0DA
:10118400053C095E0650D8A0063C0A5E0750D8A06C
:10119400073C0B5EE86AD8A0010E0E5E11D008264B
:1011A4000550D8B0053C09260650D8B0063C0A269E
:1011B4000750D8B0073C0B26E86AD8B0010E0E26BB
:1011C40003360C2ED1D70234083609360A360B36CC
:1011D4000E36045003A012D0085E0550D8A0053C7A
:1011E400095E0650D8A0063C0A5E0750D8A0073C0A
:1011F4000B5EE86AD8A0010E0E5E11D008260550D9
:10120400D8B0053C09260650D8B0063C0A2607503B
:10121400D8B0073C0B26E86AD8B0010E0E26023679
:10122400070E0C6E0234083609360A360B360E36B3
:10123400045002A012D0085E0550D8A0053C095EF7
:101244000650D8A0063C0A5E0750D8A0073C0B5EA7
:10125400E86AD8A0010E0E5E11D008260550D8B059
:10126400053C09260650D8B0063C0A260750D8B0DB
:10127400073C0B26E86AD8B0010E0E2602360C2E67
:10128400D1D70134083609360A360B360E360450E7
:1012940002A012D0085E0550D8A0053C095E065095
:1012A400D8A0063C0A5E0750D8A0073C0B5EE86A4B
:1012B400D8A0010E0E5E11D008260550D8B0053C0A
:1012C40009260650D8B0063C0A260750D8B0073C79
:1012D4000B26E86AD8B0010E0E260136070E0C6EF6
:1012E4000134083609360A360B360E36045001A08E
:1012F40012D0085E0550D8A0053C095E0650D8A05F
:10130400063C0A5E0750D8A0073C0B5EE86AD8A0EA
:10131400010E0E5E11D008260550D8B0053C0926F2
:101324000650D8B0063C0A260750D8B0073C0B2616
:10133400E86AD8B0010E0E2601360C2ED1D700343F
:10134400083609360A360B360E36045001A012D080
:10135400085E0550D8A0053C095E0650D8A0063C9E
:101364000A5E0750D8A0073C0B5EE86AD8A0010EBD
:101374000E5E11D008260550D8B0053C092606504B
:10138400D8B0063C0A260750D8B0073C0B26E86ABA
:10139400D8B0010E0E260036070E0C6E0034083647
:1013A40009360A360B360E36045000A012D0085EF9
:1013B4000550D8A0053C095E0650D8A0063C0A5E3C
:1013C4000750D8A0073C0B5EE86AD8A0010E0E5E59
:1013D40011D008260550D8B0053C09260650D8B0CF
:1013E400063C0A260750D8B0073C0B26E86AD8B05A
:1013F400010E0E2600360C2ED1D700B00ED00450AC
:1014040008260550D8B0053C09260650D8B0063C3D
:0C1414000A260750D8B0073C0B26120037
:101420000450000A08E10550000A05E1FF0E006EB5
:101430007F0E016E58D00D6A096A086A01500010CB
:10144000D8B4000C015005180A6E0ABE0D1E0B6AB6
:1014500005AE05D0041E051E042AD8B4052A01AE27
:1014600005D0001E011E002AD8B4012A0150051023
:101470000A6E0ABE10D044EC05F00BB020D00DAEC1
:10148000000C001E011E002AD8B4012A081E091EE5
:10149000082AD8B4092A000C05AE0DD001BE07D029
:1014A0000150096E0050086E016A006AE8D7016AAF
:1014B000006A002A000C011E001E0B2ADDD7082A34
:1014C000D8B4092A0450085CD8A4D9D70550095CBF
:1014D000D8A4D5D7096A086A002AD8B4012A01AE6F
:0814E000CED70000FF0C120042
:1014E800800E01015219006E800E000A005CD8B00F
:1014F8006DD152510008016E01C052F1800E0118E1
:10150800006E800E6E0A005CD8A0C0D0640E046E17
:1015180052C100F0E1EC01F0120E0024056E000E3D
:1015280000BEFF0E066E000E062205C000F006C0C3
:1015380001F0000E06BEFF0E026E036E003600902C
:10154800013602360336003600900136023603367D
:101558002F0E0024F66E490E0120F76E000E0220B1
:10156800F86E0900F5CF53F10900F5CF54F10900E1
:10157800F5CF55F10900F5CF56F1640E046E52C14E
:1015880000F0E1EC01F008C000F00A0E046EE1EC96
:1015980001F0090E0024056E000E00BEFF0E066E57
:1015A800000E062205C000F006C001F0000E06BEBF
:1015B800FF0E026E036E00360090013602360336C7
:1015C800003600900136023603362F0E0024F66EE0
:1015D800490E0120F76E000E0220F86E0900F5CFC3
:1015E80000F00900F5CF01F00900F5CF02F009007D
:1015F800F5CF03F053C104F054C105F055C106F00E
:1016080056C107F030EC02F000C053F101C054F1AC
:1016180002C055F103C056F10A0E046E52C100F023
:10162800E1EC01F008C000F000C001F0000E00BEBF
:10163800FF0E026E036E046E013601900236033609
:101648000436013601900236033604362F0E012483
:10165800F66E490E0220F76E000E0320F86E0900A0
:10166800F5CF00F00900F5CF01F00900F5CF02F041
:101678000900F5CF03F053C104F054C105F055C17A
:1016880006F056C107F030EC02F007D2800E0A0AC5
:10169800006E800E5219005C71E20A0E046E52C18F
:1016A80000F0E1EC01F0090E0024056E000E00BE0A
:1016B800FF0E066E000E062205C000F006C001F0FF
:1016C800000E06BEFF0E026E036E00360090013655
:1016D80002360336003600900136023603362F0EE6
:1016E8000024F66E490E0120F76E000E0220F86EF7
:1016F8000900F5CF53F10900F5CF54F10900F5CFF2
:1017080055F10900F5CF56F10A0E046E52C100F0EA
:10171800E1EC01F008C000F000C001F0000E00BECE
:10172800FF0E026E036E046E013601900236033618
:101738000436013601900236033604362F0E012492
:10174800F66E490E0220F76E000E0320F86E0900AF
:10175800F5CF00F00900F5CF01F00900F5CF02F050
:101768000900F5CF03F053C104F054C105F055C189
:1017780006F056C107F030EC02F08FD152C100F0EC
:10178800000E52BFFF0E016E026E036E003600900F
:10179800013602360336003600900136023603362B
:1017A8002F0E0024F66E490E0120F76E000E02205F
:1017B800F86E0900F5CF00F00900F5CF01F0090037
:1017C800F5CF02F00900F5CF03F067D1800E52196A
:1017D800006E800E6E0A005CD8A0C0D0640E046E45
:1017E80052C100F0E1EC01F0120E0024056E000E6B
:1017F80000BEFF0E066E000E062205C000F006C0F1
:1018080001F0000E06BEFF0E026E036E0036009059
:1018180001360236033600360090013602360336AA
:10182800FB0E0024F66E480E0120F76E000E022013
:10183800F86E0900F5CF53F10900F5CF54F109000E
:10184800F5CF55F10900F5CF56F1640E046E52C17B
:1018580000F0E1EC01F008C000F00A0E046EE1ECC3
:1018680001F0090E0024056E000E00BEFF0E066E84
:10187800000E062205C000F006C001F0000E06BEEC
:10188800FF0E026E036E00360090013602360336F4
:1018980000360090013602360336FB0E0024F66E41
:1018A800480E0120F76E000E0220F86E0900F5CFF1
:1018B80000F00900F5CF01F00900F5CF02F00900AA
:1018C800F5CF03F053C104F054C105F055C106F03B
:1018D80056C107F030EC02F000C053F101C054F1DA
:1018E80002C055F103C056F10A0E046E52C100F051
:1018F800E1EC01F008C000F000C001F0000E00BEED
:10190800FF0E026E036E046E013601900236033636
:10191800043601360190023603360436FB0E0124E4
:10192800F66E480E0220F76E000E0320F86E0900CE
:10193800F5CF00F00900F5CF01F00900F5CF02F06E
:101948000900F5CF03F053C104F054C105F055C1A7
:1019580006F056C107F030EC02F09FD0800E0A0A5C
:10196800006E800E5219005C71E20A0E046E52C1BC
:1019780000F0E1EC01F0090E0024056E000E00BE37
:10198800FF0E066E000E062205C000F006C001F02C
:10199800000E06BEFF0E026E036E00360090013682
:1019A8000236033600360090013602360336FB0E47
:1019B8000024F66E480E0120F76E000E0220F86E25
:1019C8000900F5CF53F10900F5CF54F10900F5CF1F
:1019D80055F10900F5CF56F10A0E046E52C100F018
:1019E800E1EC01F008C000F000C001F0000E00BEFC
:1019F800FF0E026E036E046E013601900236033646
:101A0800043601360190023603360436FB0E0124F3
:101A1800F66E480E0220F76E000E0320F86E0900DD
:101A2800F5CF00F00900F5CF01F00900F5CF02F07D
:101A38000900F5CF03F053C104F054C105F055C1B6
:101A480006F056C107F030EC02F027D052C100F082
:101A5800000E52BFFF0E016E026E036E003600903C
:101A68000136023603360036009001360236033658
:101A7800FB0E0024F66E480E0120F76E000E0220C1
:101A8800F86E0900F5CF00F00900F5CF01F0090064
:0C1A9800F5CF02F00900F5CF03F01200BA
:101AA4000450000A12E10550000A0FE10650000A32
:101AB4000CE10750000A09E1FF0E006EFF0E016EF3
:101AC4007F0E026EFF0E036EA8D0086A096A0750E3
:101AD400D8B4FDEF0DF00350D8B402EF0EF002506D
:101AE40006180A6E028E068E0E6A02C008F001C045
:101AF4000CF000C00DF004500D5E0550D8A0053C5C
:101B04000C5E0650D8A0063C085E086A0C6A0D6A92
:101B1400D8A094EF0DF0D89002320132003208328E
:101B2400010E0E6E0750035ED8A0A1EF0DF07E0EDD
:101B34000E240326D8B007EF0EF0A7EF0DF07E0EAB
:101B44000E240326D8A00CEF0EF0180E0B6E0D36E3
:101B54000C3608360036013602360E360450005E66
:101B64000550D8A0053C015E0650D8A0063C025E94
:101B740006340E120EA0C2EF0DF00D80CDEF0DF065
:101B8400045000260550D8B0053C01260650D8B0B4
:101B9400062802260D900B2EA9EF0DF0F3EF0DF0A1
:101BA400D8900036013602360E360450005E0550D9
:101BB400D8A0053C015E0650D8A0063C025E06345F
:101BC4000E10010B0D26D8B00C2AD8B4082AD8A4BC
:101BD400F3EF0DF008320C320D32032AD8B407EFBC
:101BE4000EF00AAE089E0850026E0C50016E0D50A5
:101BF400006E0FEF0EF0010EDDEC01F00FEF0EF0B2
:101C0400020E93EC00F00FEF0EF0040EA7EC00F0C0
:0C1C14000FEF0EF0080EB3EC00F0120011
:101C20000A6A0350D8A40A800750D8A40A820A502E
:101C3000D8B473EF0EF0030AD8B42CEF0EF00AB04C
:101C400027EF0EF006AE71EF0EF06FEF0EF002AE62
:101C50006FEF0EF071EF0EF00250800B0A6E029ED5
:101C60000650800B069E0A18D8B43DEF0EF00A50BD
:101C7000D8B46FEF0EF071EF0EF00750035CD8B4DC
:101C800047EF0EF0D8A063EF0EF069EF0EF00650AC
:101C9000025CD8B451EF0EF0D8A063EF0EF069EFFC
:101CA0000EF00550015CD8B45BEF0EF0D8A063EFE6
:101CB0000EF069EF0EF00450005CD8B473EF0EF034
:101CC000D8B069EF0EF00A52D8B471EF0EF06FEF92
:101CD0000EF00A52D8B46FEF0EF071EF0EF0D8800C
:0E1CE0001200D8901200D880D8841200120092
:101CEE000B6A0A6A096A00500402F4CF09F0F3CFB6
:101CFE0008F001500502F4CF0BF0F3CF0AF00050BC
:101D0E000502F3500926F4500A22E86A0B2201500C
:101D1E000402F3500926F4500A22E86A0B2208C086
:101D2E0000F009C001F00AC002F00BC003F012006F
:101D3E0001015251390806E3300E525D03E3010EE4
:081D4E00006E01D0006A1200D2
:101D56000050086E0150006E0250016E0350026E74
:101D6600036A0B6A0C6A9E0E036E0A6A020E0C6EFA
:061D7600C4EC00F01200B5
:101D7C00F00E01012A15006E0086008000C02BF1C8
:101D8C003DC052F1040E0010536F50EC06F00D0ED6
:101D9C000D6E0D2EFED73DC052F1FB0E01012B1521
:101DAC00536F50EC06F00D0E0D6E0D2EFED72AC1A2
:101DBC0000F000360090003600900036009000369F
:101DCC000090F00E00160086008000C02BF13DC084
:101DDC0052F1040E00100101536F50EC06F00D0E81
:101DEC000D6E0D2EFED73DC052F1FB0E01012B15D1
:101DFC00536F50EC06F0210E0D6E0D2EFED7120017
:101E0C0001014A6B4B6B3E6B3F6B2CC100F02DC13B
:101E1C0001F02EC102F0010E2C27000E2D232E23D3
:101E2C0000C0F6FF01C0F7FF02C0F8FF0900F5CFB4
:101E3C0000F000C03BF10052D8B40EEF1FF03B5144
:101E4C00250A0BE02AC1E1FF2BC1E2FF3BC1E6FFF3
:101E5C002A4B2B2B4A4B4B2BD8D73C6B3D6B3E6BF9
:101E6C003F6B23D03E87010E2C27000E2D232E23F3
:101E7C0059D03E81010E2C27000E2D232E2352D03B
:101E8C003E83010E2C27000E2D232E234BD03F8793
:101E9C00010E2C27000E2D232E2344D03E85010E3F
:101EAC002C27000E2D232E233DD02CC1F6FF2DC147
:101EBC00F7FF2EC1F8FF0900F5CF01F001502D0AF4
:101ECC00D1E02CC1F6FF2DC1F7FF2EC1F8FF0900A0
:101EDC00F5CF01F00150200ACCE02CC1F6FF2DC14A
:101EEC00F7FF2EC1F8FF0900F5CF01F001502B0AC6
:101EFC00C7E02CC1F6FF2DC1F7FF2EC1F8FF09007A
:101F0C00F5CF01F00150230AC2E02CC1F6FF2DC120
:101F1C00F7FF2EC1F8FF0900F5CF01F00150300A90
:101F2C00BDE001D09ED73EA301D03E913EA701D08B
:101F3C003E952CC1F6FF2DC1F7FF2EC1F8FF09000D
:101F4C00F5CF00F0000E016E00C052F1F2DE00522F
:101F5C0034E03C6B3D6B3CC100F03DC101F00A0E1E
:101F6C00046E000E056EBDDE2CC1F6FF2DC1F7FF11
:101F7C002EC1F8FF0900F5CF02F0025000243C6F8F
:101F8C00000E01203D6F300E3C5F000E3D5B010EDC
:101F9C002C27000E2D232E232CC1F6FF2DC1F7FF6D
:101FAC002EC1F8FF0900F5CF00F0000E016E00C045
:101FBC0052F1BFDE0052CFE133D02CC1F6FF2DC160
:101FCC00F7FF2EC1F8FF0900F5CF01F001502A0AE6
:101FDC0027E12FC1E9FF30C1EAFFEECF00F0EECFD1
:101FEC0001F000C0E9FF01C0EAFFEECF3CF1EECFFB
:101FFC003DF12FC1E9FF30C1EAFF020EEE24006E65
:10200C00000EEE20016E2FC1E1FF30C1E2FF00C0D7
:10201C00E6FF01C0E6FF010E2C27000E2D232E2318
:10202C002CC1F6FF2DC1F7FF2EC1F8FF0900F5CF2B
:10203C0001F001502E0A6EE1010E2C27000E2D230B
:10204C002E232CC1F6FF2DC1F7FF2EC1F8FF09007E
:10205C00F5CF01F001502A0A28E12FC1E9FF30C168
:10206C00EAFFEECF00F0EECF01F000C0E9FF01C0B7
:10207C00EAFFEECF39F1EECF3AF12FC1E9FF30C1D3
:10208C00EAFF020EEE24006E000EEE20016E2FC150
:10209C00E1FF30C1E2FF00C0E6FF01C0E6FF010E28
:1020AC002C27000E2D232E2334D0396B3A6B2CC1E8
:1020BC00F6FF2DC1F7FF2EC1F8FF0900F5CF00F098
:1020CC00000E016E00C052F134DE005222E039C124
:1020DC0000F03AC101F00A0E046E000E056E01DE2E
:1020EC002CC1F6FF2DC1F7FF2EC1F8FF0900F5CF6B
:1020FC0002F002500024396F000E01203A6F300EAE
:10210C00395F000E3A5B010E2C27000E2D232E2377
:10211C00CED703D0396B3A6B3F892CC100F02DC15F
:10212C0001F02EC102F0010E2C27000E2D232E23C0
:10213C0000C0F6FF01C0F7FF02C0F8FF0900F5CFA1
:10214C003BF1F9D04AC100F04BC101F012EF1FF086
:10215C003E89E3D73F852ED13E8B3F812BD13F83E8
:10216C0029D13E8D27D126D13E8B3E8F23D12FC135
:10217C00E9FF30C1EAFFEECF00F0EECF01F000C076
:10218C00E9FF01C0EAFFEECF46F1EECF47F12FC1D8
:10219C00E9FF30C1EAFF020EEE24006E000EEE20C5
:1021AC00016E2FC1E1FF30C1E2FF00C0E6FF01C0AC
:1021BC00E6FF000E471902E1000E461904E1190E64
:1021CC00466F000E476F486B496B48514625E96EC8
:1021DC0049514721EA6EEE520BE0010E4825006E84
:1021EC00000E4921016E00C048F101C049F1EDD744
:1021FC0039513A110AE049513A5D02E14851395DD1
:10220C0004E239C148F13AC149F13D51495D02E15D
:10221C003C51485D05E248513C5F49513D5B02D061
:10222C003C6B3D6B3EB716D03CC100F03DC101F09C
:10223C00010E3C5F000E3D5B005001100BE02AC10B
:10224C00E1FF2BC1E2FF200EE66E2A4B2B2B4A4BF3
:10225C004B2BEAD748C102F049C103F0010E485D8F
:10226C00006E000E4959016E00C048F101C049F1E1
:10227C000250031019E046C1E9FF47C1EAFF2AC129
:10228C00E1FF2BC1E2FFEECFE6FF2A4B2B2B010E19
:10229C004625006E000E4721016E00C046F101C0BC
:1022AC0047F14A4B4B2BD6D73EA716D03CC100F07A
:1022BC003DC101F0010E3C5F000E3D5B0050011072
:1022CC000BE02AC1E1FF2BC1E2FF200EE66E2A4B88
:1022DC002B2B4A4B4B2BEAD798D52FC1E9FF30C19A
:1022EC00EAFFEECF00F0EECF01F000C0E9FF01C035
:1022FC00EAFFEECF3BF12FC1E9FF30C1EAFF020E3E
:10230C00EE24006E000EEE20016E2FC1E1FF30C1F5
:10231C00E2FF00C0E6FF01C0E6FF3B0E466F010E78
:10232C00476F010E486F000E496F62D7C00E3E1307
:10233C00000E3F133FD03B51000AD8B403D73B519A
:10234C006C0AD8B405D73B514C0AD8B401D73B51D1
:10235C00660AD8B4FFD63B51450AD8B4FDD63B51DA
:10236C00650AD8B4FAD63B51670AD8B4F8D63B51B3
:10237C006F0AD8B4F6D63B51640AD8B4F4D63B51A4
:10238C00690AD8B4F0D63B51700AD8B4EDD63B519B
:10239C00580AD8B4E9D63B51780AD8B4E6D63B51A2
:1023AC00730AD8B4E4D63B51630A97E03B51750AE3
:1023BC00BDE0B3D7000E3E15006E3F51070B016E0A
:1023CC0000500110D8B4B5EF1AF03FA904D0060E96
:1023DC00396F000E3A6F2FC1E9FF30C1EAFFEECF23
:1023EC0000F0EECF01F000C0E9FF01C0EAFFEECF34
:1023FC0040F1EECF41F1EECF42F1EECF43F12FC1E0
:10240C00E9FF30C1EAFF040EEE24006E000EEE2050
:10241C00016E2FC1E1FF30C1E2FF00C0E6FF01C039
:10242C00E6FF046A056A066A076A40C100F041C10A
:10243C0001F042C102F043C103F010EC0EF0010EAA
:10244C00D8B0000E006E005205E0427F030E3E1322
:10245C00000E3F13446B456B40C100F041C101F0CD
:10246C0042C102F043C103F0046A056A066A076AB6
:10247C0083EC08F0000ED8A4010E006E0052D8B404
:10248C0089D043C100F0016A026A036AFF0E00168C
:10249C00000E01167E0E005E000E015A00C044F1C3
:1024AC0001C045F1010E005E000E015A00C044F15E
:1024BC0001C045F1030E046E000E056E12DC00C067
:1024CC0044F101C045F10A0E046E000E056E10ECCD
:1024DC000AF000C044F101C045F1800E0118026EF3
:1024EC00800E025C02E1000E005C05E2010E0101AF
:1024FC00445F000E455B010144510008526F74ECBF
:10250C000AF040C104F041C105F042C106F043C1DC
:10251C0007F030EC02F000C046F101C047F102C0F8
:10252C0048F103C049F1000E046E000E056E000E5A
:10253C00066E7F0E076E46C100F047C101F048C120
:10254C0002F049C103F010EC0EF0010ED8B0000EF1
:10255C00006E005205E0010E445F000E455B1AD080
:10256C00000E046E000E056E200E066E820E076EB7
:10257C0046C100F047C101F048C102F049C103F067
:10258C0010EC0EF0000ED8B0010E006E005202E0FE
:10259C00444B452B800E006E800E4519005C02E109
:1025AC004451000803E3010E3B6F02D044C13BF1E0
:1025BC003FB118D03FA315D0800E4519006E7F0E89
:1025CC00005C02E1FC0E445D0BE3800E4519006ECD
:1025DC00800E3A19005C02E13951445D01E201D0F0
:1025EC0001D0EFD339513A1106E03FA304D0010ECC
:1025FC00395F000E3A5B3A51000802E13951080884
:10260C0003E2080E3B6F02D039C13BF140C100F030
:10261C0041C101F042C102F043C103F0046A056AF2
:10262C00066A076A83EC08F0000ED8A4010E006E4F
:10263C000052D8B44BD144C152F174EC0AF000C032
:10264C0004F001C005F002C006F003C007F040C161
:10265C0000F041C101F042C102F043C103F052EC61
:10266C000DF000C040F101C041F102C042F103C0C5
:10267C0043F101013B510008526F74EC0AF000C0A9
:10268C0004F001C005F002C006F003C007F040C121
:10269C0000F041C101F042C102F043C103F052EC21
:1026AC000DF000C04CF101C04DF102C04EF103C061
:1026BC004FF14CC140F14DC141F14EC142F14FC1FE
:1026CC0043F14CC100F04DC101F04EC102F04FC1BD
:1026DC0003F0E7EC07F0ABEC0EF000C004F001C027
:1026EC0005F002C006F003C007F04CC100F04DC16C
:1026FC0001F04EC102F04FC103F063EC06F0000E86
:10270C00046E000E056E000E066E7E0E076E10EC4B
:10271C000EF0000ED8B0010E006E00521AE040C14F
:10272C0000F041C101F042C102F043C103F0000EC0
:10273C00046E000E056E000E066E7E0E076ECEEC5D
:10274C0002F000C040F101C041F102C042F103C0EF
:10275C0043F140C100F041C101F042C102F043C15C
:10276C0003F0E7EC07F001013B51010F096E0A6A17
:10277C00000E0A2209C004F00AC005F0000E0ABEC1
:10278C00FF0E066E076E04360490053606360736C5
:10279C0004360490053606360736400E0424F66ED1
:1027AC004B0E0520F76E000E0620F86E0900F5CFD3
:1027BC0005F00900F5CF06F00900F5CF07F0090088
:1027CC00F5CF08F00850035C08E10750025C05E106
:1027DC000650015C02E10550005C1EE3010140C1A2
:1027EC0000F041C101F042C102F043C103F0CD0E33
:1027FC00046ECC0E056E4C0E066E7B0E076E30EC26
:10280C0002F000C040F101C041F102C042F103C02E
:10281C0043F1444B452B5AD040C100F041C101F06B
:10282C0042C102F043C103F0E7EC07F03BC104F0F6
:10283C00000E056E066E076E0436049005360636DD
:10284C00073604360490053606360736400E042447
:10285C00F66E4B0E0520F76E000E0620F86E090082
:10286C00F5CF05F00900F5CF06F00900F5CF07F01C
:10287C000900F5CF08F00850035C08E10750025C32
:10288C0005E10650015C02E10550005C1FE201010C
:10289C0040C100F041C101F042C102F043C103F05C
:1028AC00000E046E000E056E200E066E820E076E74
:1028BC0030EC02F000C040F101C041F102C042F125
:1028CC0003C043F1010E445F000E455B01013FA3C1
:1028DC0093D03FB791D0800E000A006E800E3A194B
:1028EC00005C02E139510A0804E20A0E396F000E4D
:1028FC003A6F40C100F041C101F042C102F043C146
:10290C0003F0E7EC07F000C046F101C047F102C04C
:10291C0048F103C049F1465147114811491142E0B1
:10292C000A0E046E000E056E066E076E46C100F0B0
:10293C0047C101F048C102F049C103F09AEC08F01C
:10294C0008C000F009C001F00AC002F00BC003F08F
:10295C00000E046E031808E10450021805E104503F
:10296C00011802E10050000A1DE1010E395F000E52
:10297C003A5B0A0E046E000E056E066E076E46C1BB
:10298C0000F047C101F048C102F049C103F09AECD4
:10299C0008F000C046F101C047F102C048F103C085
:1029AC0049F1B9D7800E3A19006E800E005C02E135
:1029BC003B51395D21E239513B5D526F74EC0AF0A9
:1029CC0000C004F001C005F002C006F003C007F01F
:1029DC0040C100F041C101F042C102F043C103F01B
:1029EC0052EC0DF000C040F101C041F102C042F1C7
:1029FC0003C043F139C13BF1050E01013925006ECD
:102A0C00000E3A21016E00503C5F01503D5B395184
:102A1C003A1103E13FB701D004D0010E3C5F000E28
:102A2C003D5B030E3E15006E3FC101F0000E01161A
:102A3C000050011004E0010E3C5F000E3D5B3EA512
:102A4C0039D03EA312D03EA103D02D0E316F02D04F
:102A5C002B0E316F2AC1E1FF2BC1E2FF31C1E6FF22
:102A6C002A4B2B2B4A4B4B2B0CD03EA10AD02AC104
:102A7C00E1FF2BC1E2FF200EE66E2A4B2B2B4A4BBB
:102A8C004B2B800E006E800E3D19005C02E13C5118
:102A9C0000080FE22AC1E1FF2BC1E2FF300EE66E07
:102AAC002A4B2B2B4A4B4B2B010E3C5F000E3D5BF4
:102ABC00E8D73AD03EB718D0800E006E800E3D1984
:102ACC00005C02E13C5100080FE22AC1E1FF2BC17E
:102ADC00E2FF200EE66E2A4B2B2B4A4B4B2B010EA2
:102AEC003C5F000E3D5BE8D73EA312D03EA103D065
:102AFC002D0E326F02D02B0E326F2AC1E1FF2BC18B
:102B0C00E2FF32C1E6FF2A4B2B2B4A4B4B2B0CD04E
:102B1C003EA10AD02AC1E1FF2BC1E2FF200EE66ED6
:102B2C002A4B2B2B4A4B4B2B40C100F041C101F0DF
:102B3C0042C102F043C103F0E7EC07F000C046F1DC
:102B4C0001C047F102C048F103C049F13BC100F09C
:102B5C00000E016E026E036E0036009001360236D6
:102B6C00033600360090013602360336400E002440
:102B7C00F66E4B0E0120F76E000E0220F86E090067
:102B8C00F5CF04F00900F5CF05F00900F5CF06F0FC
:102B9C000900F5CF07F046C100F047C101F048C16C
:102BAC0002F049C103F09AEC08F0300E00262AC15D
:102BBC00E1FF2BC1E2FF00C0E6FF2A4B2B2B4A4B57
:102BCC004B2B39513A1103E13FB701D06FD02AC1D9
:102BDC00E1FF2BC1E2FF2E0EE66E2A4B2B2B4A4B4C
:102BEC004B2B3B51395F000E3A5B3B534DE03B079F
:102BFC003BC100F0000E016E026E036E00360090B9
:102C0C0001360236033600360090013602360336A2
:102C1C00400E0024F66E4B0E0120F76E000E0220C3
:102C2C00F86E0900F5CF04F00900F5CF05F00900A6
:102C3C00F5CF06F00900F5CF07F046C100F047C10B
:102C4C0001F048C102F049C103F09AEC08F00A0EF9
:102C5C00046E000E056E066E076E9AEC08F008C046
:102C6C0000F009C001F00AC002F00BC003F0300EF6
:102C7C0000262AC1E1FF2BC1E2FF00C0E6FF2A4B70
:102C8C002B2B4A4B4B2BB1D739513A110FE02AC1A0
:102C9C00E1FF2BC1E2FF300EE66E2A4B2B2B4A4B89
:102CAC004B2B010E395F000E3A5BEED73EAB0BD0CF
:102CBC002AC1E1FF2BC1E2FF450EE66E2A4B2B2BFE
:102CCC004A4B4B2B0AD02AC1E1FF2BC1E2FF650E08
:102CDC00E66E2A4B2B2B4A4B4B2B800E4519006E64
:102CEC00800E005C02E1000E445D11E244510008CC
:102CFC00446F4551000E45572AC1E1FF2BC1E2FF3D
:102D0C002D0EE66E2A4B2B2B4A4B4B2B0AD02AC18D
:102D1C00E1FF2BC1E2FF2B0EE66E2A4B2B2B4A4B0D
:102D2C004B2B0A0E046E000E056E44C100F045C11B
:102D3C0001F010EC0AF0300E00262AC1E1FF2BC185
:102D4C00E2FF00C0E6FF01012A4B2B2B4A4B4B2B19
:102D5C000A0E046E000E056E44C100F045C101F070
:102D6C0010EC0AF008C000F009C001F0300E00268B
:102D7C002AC1E1FF2BC1E2FF00C0E6FF01012A4B93
:102D8C002B2B4A4B4B2B3EA71AD0800E006E800E7D
:102D9C003D19005C02E13C51000811E22AC1E1FF3F
:102DAC002BC1E2FF200EE66E2A4B2B2B4A4B4B2BF2
:102DBC00010E3C5F000E3D5B3C513D11EFE10BEF12
:102DCC000FF03FA3F3D0800E4519006E800E005C0F
:102DDC0002E1000E445D0AE2010E445D006E000E3D
:102DEC004559016E0050395F01503A5B40C100F00B
:102DFC0041C101F042C102F043C103F0E7EC07F01E
:102E0C0000C046F101C047F102C048F103C049F1CE
:102E1C00010E3B6F3B510A0A34E03BC100F0000E3F
:102E2C00016E026E036E00360090013602360336D8
:102E3C0000360090013602360336400E0024F66E42
:102E4C004B0E0120F76E000E0220F86E0900F5CF34
:102E5C0001F00900F5CF02F00900F5CF03F00900ED
:102E6C00F5CF04F00450495D08E10350485D05E1DD
:102E7C000250475D02E10150465D01E202D03B2B5E
:102E8C00C9D73B51395D506F000E3A59516F50C143
:102E9C0039F151C13AF146C100F047C101F048C1C6
:102EAC0002F049C103F0ABEC0EF000C004F001C01D
:102EBC0005F002C006F003C007F040C100F041C1AC
:102ECC0001F042C102F043C103F063EC06F000C014
:102EDC004CF101C04DF102C04EF103C04FF150C195
:102EEC0052F174EC0AF04CC104F04DC105F04EC126
:102EFC0006F04FC107F030EC02F0000E046E000E2D
:102F0C00056E000E066E7E0E076ECEEC02F0E7EC40
:102F1C0007F000C046F101C047F102C048F103C000
:102F2C0049F139513A1142E00A0E046E000E056E59
:102F3C00066E076E46C100F047C101F048C102F0B1
:102F4C0049C103F09AEC08F008C000F009C001F088
:102F5C000AC002F00BC003F0000E046E031808E167
:102F6C000450021805E10450011802E10050000A57
:102F7C001DE10A0E046E000E056E066E076E46C14C
:102F8C0000F047C101F048C102F049C103F09AECCE
:102F9C0008F000C046F101C047F102C048F103C07F
:102FAC0049F1010E395F000E3A5BBBD7800E006E03
:102FBC00800E3A19005C02E139510C0816E339C154
:102FCC0052F166EC06F040C104F041C105F042C17B
:102FDC0006F043C107F0CEEC02F000C040F101C096
:102FEC0041F102C042F103C043F140C100F041C1C4
:102FFC0001F042C102F043C103F0046A056A066A9B
:10300C00076A83EC08F0000ED8A4010E006E005283
:10301C00D8B477D040C100F041C101F042C102F0F8
:10302C0043C103F0E7EC07F0000E046E031808E14F
:10303C000450021805E10450011802E10050000A86
:10304C0060E1800E006E800E4519005C02E1445177
:10305C00010857E244C152F174EC0AF000C004F0CC
:10306C0001C005F002C006F003C007F040C100F03B
:10307C0041C101F042C102F043C103F052EC0DF02A
:10308C005F0E046E700E056E090E066E810E076ED5
:10309C0010EC0EF0010ED8B0000E006E005206E0DF
:1030AC00090E0101445F000E455B05D00101080EBD
:1030BC00445F000E455B44C152F174EC0AF000C051
:1030CC0004F001C005F002C006F003C007F040C1D7
:1030DC0000F041C101F042C102F043C103F052ECD7
:1030EC000DF0E7EC07F000C046F101C047F102C05B
:1030FC0048F103C049F10101406B416B426B436BDA
:10310C0038D040C100F041C101F042C102F043C1CE
:10311C0003F0E7EC07F000C046F101C047F102C034
:10312C0048F103C049F146C100F047C101F048C164
:10313C0002F049C103F0ABEC0EF000C004F001C08A
:10314C0005F002C006F003C007F040C100F041C119
:10315C0001F042C102F043C103F063EC06F000C081
:10316C0040F101C041F102C042F103C043F1446B94
:10317C00456B010E3B6F3B510A0A34E03BC100F03A
:10318C00000E016E026E036E0036009001360236A0
:10319C00033600360090013602360336400E00240A
:1031AC00F66E4B0E0120F76E000E0220F86E090031
:1031BC00F5CF01F00900F5CF02F00900F5CF03F0CF
:1031CC000900F5CF04F00450495D08E10350485D57
:1031DC0005E10250475D02E10150465D01E202D07B
:1031EC003B2BC9D73B513925006E000E3A21016E9D
:1031FC00445100264551012200503C5F01503D5B7B
:10320C003FB704D039513A1101E104D0010E3C5FB3
:10321C00000E3D5B030E3E15006E3FC101F0000E2B
:10322C0001160050011004E0010E3C5F000E3D5BE6
:10323C003EA539D03EA312D03EA103D02D0E336F44
:10324C0002D02B0E336F2AC1E1FF2BC1E2FF33C139
:10325C00E6FF2A4B2B2B4A4B4B2B0CD03EA10AD012
:10326C002AC1E1FF2BC1E2FF200EE66E2A4B2B2B6D
:10327C004A4B4B2B800E006E800E3D19005C02E118
:10328C003C5100080FE22AC1E1FF2BC1E2FF300ED6
:10329C00E66E2A4B2B2B4A4B4B2B010E3C5F000E40
:1032AC003D5BE8D73AD03EB718D0800E006E800E4A
:1032BC003D19005C02E13C5100080FE22AC1E1FF1C
:1032CC002BC1E2FF200EE66E2A4B2B2B4A4B4B2BCD
:1032DC00010E3C5F000E3D5BE8D73EA312D03EA131
:1032EC0003D02D0E346F02D02B0E346F2AC1E1FFA8
:1032FC002BC1E2FF34C1E6FF2A4B2B2B4A4B4B2B45
:10330C000CD03EA10AD02AC1E1FF2BC1E2FF200E56
:10331C00E66E2A4B2B2B4A4B4B2B3BC100F03B0749
:10332C0000524CE03BC100F0000E016E026E036EC9
:10333C000036009001360236033600360090013616
:10334C0002360336400E0024F66E4B0E0120F76E4B
:10335C00000E0220F86E0900F5CF04F00900F5CF3D
:10336C0005F00900F5CF06F00900F5CF07F046C1CE
:10337C0000F047C101F048C102F049C103F09AECDA
:10338C0008F00A0E046E000E056E066E076E9AECBF
:10339C0008F008C000F009C001F00AC002F00BC030
:1033AC0003F0300E00262AC1E1FF2BC1E2FF00C062
:1033BC00E6FF2A4B2B2B4A4B4B2BAFD7800E006EC4
:1033CC00800E4519005C02E1445100080FE22AC14D
:1033DC00E1FF2BC1E2FF300EE66E2A4B2B2B4A4B42
:1033EC004B2B010E445F000E455BE8D7800E000AA4
:1033FC00006E800E3A19005C02E13951080803E2B4
:10340C00080E3B6F02D039C13BF13B51395F000EC6
:10341C003A5B3B5303E13FB701D00AD02AC1E1FF2D
:10342C002BC1E2FF2E0EE66E2A4B2B2B4A4B4B2B5D
:10343C003BC152F174EC0AF040C104F041C105F0FB
:10344C0042C106F043C107F030EC02F0B8EC05F0D5
:10345C0000C046F101C047F102C048F103C049F178
:10346C003B534DE03B073BC100F0000E016E026E7A
:10347C00036E00360090013602360336003600909B
:10348C00013602360336400E0024F66E4B0E012038
:10349C00F76E000E0220F86E0900F5CF04F009005B
:1034AC00F5CF05F00900F5CF06F00900F5CF07F0D0
:1034BC0046C100F047C101F048C102F049C103F018
:1034CC009AEC08F00A0E046E000E056E066E076E7E
:1034DC009AEC08F008C000F009C001F00AC002F034
:1034EC000BC003F0300E00262AC1E1FF2BC1E2FF16
:1034FC0000C0E6FF2A4B2B2B4A4B4B2BB1D7395133
:10350C003A110FE02AC1E1FF2BC1E2FF300EE66E4B
:10351C002A4B2B2B4A4B4B2B010E395F000E3A5B7F
:10352C00EED73EA71AD0800E006E800E3D19005CBF
:10353C0002E13C51000811E22AC1E1FF2BC1E2FF7C
:10354C00200EE66E2A4B2B2B4A4B4B2B010E3C5F6D
:10355C00000E3D5B3C513D11EFE10BEF0FF0C00E47
:10356C003E15016E3FC102F0000E0216000E02184D
:10357C0002E1000E0118D8A480D03EA927D02FC19B
:10358C00E9FF30C1EAFFEECF00F0EECF01F000C052
:10359C00E9FF01C0EAFFEECF46F1EECF47F1EECFE7
:1035AC0048F1EECF49F12FC1E9FF30C1EAFF040E1B
:1035BC00EE24006E000EEE20016E2FC1E1FF30C133
:1035CC00E2FF00C0E6FF01C0E6FF2FD02FC1E9FFEC
:1035DC0030C1EAFFEECF00F0EECF01F000C0E9FF02
:1035EC0001C0EAFFEECF00F0EECF01F0000E01BEFD
:1035FC00FF0E026E036E00C046F101C047F102C01F
:10360C0048F103C049F12FC1E9FF30C1EAFF020EB6
:10361C00EE24006E000EEE20016E2FC1E1FF30C1D2
:10362C00E2FF00C0E6FF01C0E6FF800E4919006E04
:10363C00800E005C08E1000E485D05E1000E475D60
:10364C0002E1000E465D18E2030E3E13000E3F131E
:10365C00006A016A026A036A4651005E4751015AC8
:10366C004851025A4951035A00C046F101C047F172
:10367C0002C048F103C049F14ED03EA927D02FC15A
:10368C00E9FF30C1EAFFEECF00F0EECF01F000C051
:10369C00E9FF01C0EAFFEECF46F1EECF47F1EECFE6
:1036AC0048F1EECF49F12FC1E9FF30C1EAFF040E1A
:1036BC00EE24006E000EEE20016E2FC1E1FF30C132
:1036CC00E2FF00C0E6FF01C0E6FF25D02FC1E9FFF5
:1036DC0030C1EAFFEECF00F0EECF01F000C0E9FF01
:1036EC0001C0EAFFEECF46F1EECF47F1000E486F76
:1036FC00496F2FC1E9FF30C1EAFF020EEE24006EC4
:10370C00000EEE20016E2FC1E1FF30C1E2FF00C0C0
:10371C00E6FF01C0E6FF000E3A1902E1000E39196E
:10372C000FE1000E006E491908E10050481905E13F
:10373C000050471902E14651000A02E1394B3A2B7D
:10374C00C00E3E15006E00C005F0AED0010E3B6FF2
:10375C003B510A0A34E03BC100F0000E016E026ED0
:10376C00036E0036009001360236033600360090A8
:10377C00013602360336400E0024F66E4B0E012045
:10378C00F76E000E0220F86E0900F5CF01F009006B
:10379C00F5CF02F00900F5CF03F00900F5CF04F0E6
:1037AC000450495D08E10350485D05E10250475D56
:1037BC0002E10150465D01E202D03B2BC9D782D019
:1037CC00010E3B6F3B51080A34E03BC100F0000E88
:1037DC00016E026E036E003600900136023603361F
:1037EC0000360090013602360336A90E0024F66E20
:1037FC004B0E0120F76E000E0220F86E0900F5CF7B
:10380C0001F00900F5CF02F00900F5CF03F0090033
:10381C00F5CF04F00450495D08E10350485D05E123
:10382C000250475D02E10150465D01E202D03B2BA4
:10383C00C9D748D0010E3B6F3B510C0A34E03BC159
:10384C0000F0000E016E026E036E00360090013621
:10385C000236033600360090013602360336C60EA9
:10386C000024F66E490E0120F76E000E0220F86E51
:10387C000900F5CF01F00900F5CF02F00900F5CFF2
:10388C0003F00900F5CF04F00450495D08E1035042
:10389C00485D05E10250475D02E10150465D01E2E1
:1038AC0002D03B2BC9D70ED00550000AD8B44ED746
:1038BC000550C00AD8B44AD70550800A81E005509B
:1038CC00400AB8E0800E006E800E3A19005C02E1EE
:1038DC0039513B5D03E239C13BF10DD0800E3A19F1
:1038EC00006E800E005C02E13B51395D04E23BC18D
:1038FC0039F1000E3A6F3C513D110EE0030E3E15AE
:10390C00006E3FC101F0000E01160050011004E0E2
:10391C00010E3C5F000E3D5B800E3A19006E800E6E
:10392C003D19005C02E13C51395D05E239513C5FC7
:10393C003A513D5B02D03C6B3D6BC40E3E15016EA3
:10394C003F51080B026E0250080A02E1400E0118AA
:10395C0008E13C513D1104E0010E3C5F000E3D5B63
:10396C001CD0C00E3E15016E3F51080B026E02506A
:10397C00080A02E1800E011810E1800E006E800E24
:10398C003D19005C02E13C51020805E2020E3C5F6D
:10399C00000E3D5B02D03C6B3D6B3EA55DD03EA363
:1039AC0012D03EA103D02D0E356F02D02B0E356FE9
:1039BC002AC1E1FF2BC1E2FF35C1E6FF2A4B2B2BBD
:1039CC004A4B4B2B34D03EA10BD02AC1E1FF2BC16B
:1039DC00E2FF200EE66E2A4B2B2B4A4B4B2B27D0AB
:1039EC00C00E3E15016E3F51080B026E0250080AC4
:1039FC0002E1800E01181BE12AC1E1FF2BC1E2FF9D
:103A0C00300EE66E2A4B2B2B4A4B4B2B3EAB03D086
:103A1C00580E366F02D0780E366F2AC1E1FF2BC1DB
:103A2C00E2FF36C1E6FF2A4B2B2B4A4B4B2B3C516A
:103A3C003D1111E02AC1E1FF2BC1E2FF300EE66E11
:103A4C002A4B2B2B4A4B4B2B010E3C5F000E3D5B44
:103A5C003C513D11EFE174D03C513D1113E03EB7A8
:103A6C0011D02AC1E1FF2BC1E2FF200EE66E2A4BDA
:103A7C002B2B4A4B4B2B010E3C5F000E3D5B3C51FC
:103A8C003D11EFE13EA312D03EA103D02D0E376FB6
:103A9C0002D02B0E376F2AC1E1FF2BC1E2FF37C1D9
:103AAC00E6FF2A4B2B2B4A4B4B2B0CD03EA10AD0BA
:103ABC002AC1E1FF2BC1E2FF200EE66E2A4B2B2B15
:103ACC004A4B4B2BC00E3E15016E3F51080B026E3C
:103ADC000250080A02E1400E01180BE12AC1E1FF75
:103AEC002BC1E2FF300EE66E2A4B2B2B4A4B4B2B95
:103AFC0027D0C00E3E15016E3F51080B026E0250CE
:103B0C00080A02E1800E01181BE12AC1E1FF2BC15A
:103B1C00E2FF300EE66E2A4B2B2B4A4B4B2B3EAB67
:103B2C0003D0580E386F02D0780E386F2AC1E1FFDF
:103B3C002BC1E2FF38C1E6FF2A4B2B2B4A4B4B2BF8
:103B4C00800E006E800E3A19005C02E139513B5D2B
:103B5C000BE22AC1E1FF2BC1E2FF300EE66E2A4BCD
:103B6C002B2B4A4B4B2BECD739C100F03AC101F04F
:103B7C00010E395F000E3A5B00500110D8B42AD107
:103B8C00C00E3E15006E00C04CF10AD139C100F0D8
:103B9C003AC101F0000E3ABFFF0E026E036E003602
:103BAC00009001360236033600360090013602369C
:103BBC000336400E0024F66E4B0E0120F76E000EFD
:103BCC000220F86E0900F5CF04F00900F5CF05F0DE
:103BDC000900F5CF06F00900F5CF07F046C100F05B
:103BEC0047C101F048C102F049C103F09AEC08F05A
:103BFC000A0E046E000E056E066E076E9AEC08F047
:103C0C0008C000F009C001F00AC002F00BC003F0BC
:103C1C00300E00243B6FD3D03EAB45D039C100F001
:103C2C003AC101F0000E3ABFFF0E026E036E003671
:103C3C00009001360236033600360090013602360B
:103C4C000336A90E0024F66E4B0E0120F76E000E03
:103C5C000220F86E0900F5CF04F00900F5CF05F04D
:103C6C000900F5CF06F00900F5CF07F046C100F0CA
:103C7C0047C101F048C102F049C103F09AEC08F0C9
:103C8C000F0E0016000E011602160316A80E0024C5
:103C9C00F66E4C0E0120F76E000E0220F86E090035
:103CAC00F5CF3BF144D039C100F03AC101F0000E20
:103CBC003ABFFF0E026E036E0036009001360236DC
:103CCC00033600360090013602360336A90E002466
:103CDC00F66E4B0E0120F76E000E0220F86E0900F6
:103CEC00F5CF04F00900F5CF05F00900F5CF06F08B
:103CFC000900F5CF07F046C100F047C101F048C1FB
:103D0C0002F049C103F09AEC08F00F0E0016000EF9
:103D1C00011602160316B90E0024F66E4C0E012085
:103D2C00F76E000E0220F86E0900F5CF3BF147D07C
:103D3C0039C100F03AC101F0000E3ABFFF0E026E1D
:103D4C00036E0036009001360236033600360090C2
:103D5C00013602360336C60E0024F66E490E0120DB
:103D6C00F76E000E0220F86E0900F5CF04F0090082
:103D7C00F5CF05F00900F5CF06F00900F5CF07F0F7
:103D8C0046C100F047C101F048C102F049C103F03F
:103D9C009AEC08F0070E00143B6F300E3B270FD047
:103DAC004C51000AD8B4F2D64C51C00AD8B4EED655
:103DBC004C51800AD8B430D74C51400AB9E02AC1D2
:103DCC00E1FF2BC1E2FF3BC1E6FF2A4B2B2B4A4BF9
:103DDC004B2BCAD63EA71AD0800E006E800E3D1912
:103DEC00005C02E13C51000811E22AC1E1FF2BC149
:103DFC00E2FF200EE66E2A4B2B2B4A4B4B2B010E6F
:103E0C003C5F000E3D5B3C513D11EFE10BEF0FF0C1
:0A3E1C004AC100F04BC101F0120092
:103E2600F00E01011D15006E008600C000F13DC0B8
:103E360052F1040E0010536F50EC06F0420E0D6E58
:103E46000D2EFED700003DC052F1FB0E01010015FC
:103E5600536F50EC06F0420E0D6E0D2EFED700008D
:103E660001011E51010A2BE11DC100F00036009030
:103E7600003600900036009000360090F00E0016D6
:103E8600008600C000F13DC052F1040E0010536FD1
:103E960050EC06F00D0E0D6E0D2EFED73DC052F104
:103EA600FB0E01010015536F50EC06F01A0E0C6E56
:103EB600F80E0D6E0D2EFED70C2EFCD7000012004C
:103EC6001DC1F6FF1EC1F7FF1FC1F8FF0900F5CFA0
:103ED60000F0005212E01DC1F6FF1EC1F7FF1FC120
:103EE600F8FF0900F5CF2AF1BEEC0EF0010E010134
:0C3EF6001D27000E1E231F23E3D712001F
:103F0200220E0101286F010E296F1DC12AF11EC167
:103F12002BF11FC12CF120C12DF121C12EF1280E50
:103F22002F6F010E306F06EC0FF000C026F101C0BA
:103F320027F100501D25E16E01501E21E26EE66A56
:0A3F420026C100F027C101F01200B3
:103F4C000D0E01015D6F9AEC00F00A0E01015D6F20
:063F5C009AEC00F01200D7
:103F620001011F6B1DC1E9FF1EC1EAFFEECF00F187
:103F72000051000A0FE000C15DF19AEC00F001016E
:103F82001F2B1F511D25E96E000E1E21EA6EEECF7A
:063F920000F1EED7120061
:103F9800086A096A100E0C6E013408360936045096
:103FA800085E0550D8A0053C095ED8B007D004507B
:103FB80008260550D8B0053C0926D89000360136A9
:063FC8000C2EEAD71200E6
:103FCE0017C1F6FF18C1F7FF19C1F8FF0900F5CFA9
:103FDE0000F0005212E017C1F6FF18C1F7FF19C129
:103FEE00F8FF0900F5CF5DF19AEC00F0010E01012A
:0C3FFE001727000E18231923E3D7120028
:10400A000900F5CFE6FF0006FBE10106F9E112001F
:10401A00820E0001A06F030EA16F000EA26F000EA8
:10402A00A36FE00E0101116F0A0E126F000E136FDB
:10403A00000E146FFF0E0D6FFF0E0E6F000E0F6F46
:10404A00000E106FFF0E096FFF0E0A6FFF0E0B6F47
:10405A00FF0E0C6FC20E016F090E026F570E036F2F
:10406A00010E046F840E056F0A0E066F000E076FAD
:10407A00000E086F949894968B988B9694889486E1
:0A408A00C79EC79C380EC66E1200D8
:10409400340E246E010E256E5D0E266E010E276E03
:1040A400FF0E286EFF0E296E000E2A6E000E2B6E78
:1040B400FF0E326EFF0E336E000E346E000E356E40
:1040C4001E0E366E410E376E000E386E000E396EBF
:1040D400AC8A900EAB6E948E949C9EAA03D0AECF05
:0640E40000F0FBD7120002
:1040EA00FF0E816E830E936E0F01396B070E806E81
:1040FA00386B388138830F0E926E806A929889885D
:10410A00826A3A6B800E946E94869488948E949CFC
:04411A00606A1200C5
:0A411E00000EACB2010E006E12009C
:104128002AD0800E01011D6F010E1E6F78DEFD0E74
:1041380001011D6F4C0E1E6F000E1F6FC0DE800E3A
:1041480001011D6F010E1E6F6ADE22D0C00E010133
:104158001D6F010E1E6F63DE970E01011D6F4C0E61
:104168001E6F000E1F6FABDEC00E01011D6F010E2A
:104178001E6F55DE0DD0000E0101181902E1010E67
:104188001719CFE0000E181902E1020E1719DEE028
:02419800120013
:10419A0019C1F6FF1AC1F7FF1BC1F8FF0900F5CFD5
:1041AA0000F0005218E019C1F6FF1AC1F7FF1BC14F
:1041BA00F8FF0900F5CF00F017C1E1FF18C1E2FFCF
:1041CA0000C0E6FF0101174B182B010E1927000E3C
:1041DA001A231B23DDD717C1E1FF18C1E2FFE66AE4
:0241EA001200C1
:1041EC00200E01015D6F9AEC00F0200E01015D6F55
:1041FC009AEC00F0300E01015D6F9AEC00F0030EAA
:10420C000B6E080E0C6E770E0D6E0D2EFED70C2E4F
:10421C00FCD70B2EFAD7300E01011D6F1E6BFDDD86
:10422C00310E01015D6F9AEC00F0060E0C6E300E33
:10423C000D6E0D2EFED70C2EFCD70000300E01019A
:10424C001D6F1E6BEADD320E01015D6F9AEC00F002
:10425C00060E0C6E300E0D6E0D2EFED70C2EFCD7EE
:10426C000000300E01011D6F1E6BD7DD330E0101F6
:10427C005D6F9AEC00F01A0E0C6EF80E0D6E0D2E92
:10428C00FED70C2EFCD70000280E01011D6F010E6D
:10429C001E6FC3DD350E01015D6F9AEC00F00B0E45
:1042AC000C6E620E0D6E0D2EFED70C2EFCD7000080
:1042BC00080E01011D6F010E1E6FAFDD360E0101E0
:1042CC005D6F9AEC00F00B0E0C6E620E0D6E0D2EE7
:1042DC00FED70C2EFCD70000010E01011D6F010E44
:1042EC001E6F9BDD370E01015D6F9AEC00F0680EBE
:1042FC000C6EE40E0D6E0D2EFED70C2EFCD70000AE
:10430C00060E01011D6F010E1E6F87DD380E0101B7
:10431C005D6F9AEC00F00B0E0C6E620E0D6E0D2E96
:10432C00FED70C2EFCD700000C0E01011D6F010EE8
:10433C001E6F73DD390E01015D6F9AEC00F00D0EEE
:10434C0001015D6F9AEC00F00A0E01015D6F9AECB1
:10435C0000F00B0E0C6E620E0D6E0D2EFED70C2E99
:06436C00FCD70000120066
:104372000001FF6B70EC05F017C157F1E1EC04F09E
:1043820000521CE02CC01DF12DC01EF1F60E0101E1
:104392001F6F490E206F000E216F17C122F118C145
:1043A20023F117C124F118C125F1AADD2CC01DF19A
:1043B2002DC01EF1D5DD0001FF6B1BD02CC01DF1FD
:1043C2002DC01EF1120E01011F6F4B0E206F000E49
:1043D200216F17C122F118C123F117C124F118C1AD
:1043E20025F18EDD2CC01DF12DC01EF1B9DD17C1E6
:0E43F200FFF042EC05F0A9DDFFC000F0120064
:104400000001FF6B050EFF5D0CE2FF510101192554
:10441000E16E000E1A21E26E200EE66E0001FF2B07
:10442000F1D7FF5101011925E16E000E1A21E26E4C
:10443000E66A0001FF07FF51010119251B6F000EFD
:104440001A211C6F0A0E046E000E056E17C100F0D3
:1044500018C101F0A1DD08C000F009C001F0300E64
:1044600000261BC1E1FF1CC1E2FF00C0E6FF0A0EEF
:10447000046E000E056E17C100F018C101F08CDD4E
:1044800000C017F101C018F1000E011802E1000E82
:0E449000001801E103D00001FF07CDD7120094
:10449E000101196B1A6B17C1E9FF18C1EAFFEE5043
:1044AE00000A17E0800E1A19006E800E005C02E101
:1044BE00100E195D0EE217C1E9FF18C1EAFFEECF2B
:1044CE002AF1BEEC0EF00101174B182B194B1A2BCB
:0444DE00E2D712000F
:1044E2009DEC26F0D388D38CD38AD382D390D3B4D5
:1044F20001D0FDD7F9DD00017E6B7F6B800E7F1945
:10450200006E800E005C02E1050E7E5D21E289985C
:104512000B0E0B6E260E0C6E5D0E0D6E0D2EFED763
:104522000C2EFCD70B2EFAD70000000089880B0E48
:104532000B6E260E0C6E5D0E0D6E0D2EFED70C2E22
:10454200FCD70B2EFAD7000000007E4B7F2BD6D76C
:104552003E0E2C6E000E2D6EB886B06ACF0EAF6E78
:10456200AC8497DD030E0B6E080E0C6E770E0D6E8B
:104572000D2EFED70C2EFCD70B2EFAD7CFDD005016
:10458200010A06E10D0E01015D6F9AEC00F0F6D70B
:104592000C0E01015D6F9AEC00F0D7DCFE0E0101FA
:1045A200176F4B0E186F000E196F10DD730E01019D
:1045B200176F4C0E186F000E196F08DD950E010172
:1045C200176F490E186F000E196F00DDE40E01011E
:1045D200176F4A0E186F000E196FF8DC180E0101E2
:1045E200176F4C0E186F000E196FF0DC630E01018D
:1045F200176F490E186F000E196FE8DCC40E010127
:10460200176F480E186F000E196FE0DC5F0E010184
:10461200176F4C0E186F000E196FD8DC0A0EC86E99
:10462200FBDC0B0E0B6E260E0C6E5D0E0D6E0D2E50
:10463200FED70C2EFCD70B2EFAD700000000300E4E
:1046420000017E6F000E7F6F800E7F19006E800E5C
:10465200005C02E1800E7E5D26E27EC017F17FC023
:1046620018F186DE005000080BE2800E00017F196F
:10467200006E800E005C02E1800E7E5D01E213D0CE
:10468200020E0B6E040E0C6EBA0E0D6E00010D2E94
:10469200FDD70C2EFBD70B2EF9D70000020E7E277A
:1046A200000E7F23D1D7030E0B6E080E0C6E770E11
:1046B2000D6E0D2EFED70C2EFCD70B2EFAD77EC018
:1046C2003DF04A0E3A6EE40E0101176F4B0E186F61
:1046D200000E196F7BDC89DD38DC010E01012A6FC7
:1046E200BEEC0EF0070E0B6E170E0C6E6A0E0D6E00
:1046F2000D2EFED70C2EFCD70B2EFAD70000680E1B
:104702000101176F4B0E186F000E196F5FDC2CC082
:1047120017F12DC018F1DB0E0101196F4C0E1A6F43
:10472200000E1B6F39DD2CC01DF12DC01EF118DCEF
:104732000CDC010E0101176F000E186FF4DC860EFF
:1047420001011D6F4C0E1E6F000E1F6F63EC1FF0F8
:10475200290E0B6E960E0C6E7F0E0D6E0D2EFED771
:104762000C2EFCD70B2EFAD7890E0101176F4B0EB8
:10477200186F000E196F2ADC2CC017F12DC018F12A
:10478200CA0E0101196F4C0E1A6F000E1B6F04DD69
:104792002CC01DF12DC01EF1B1EC1FF0A6EC1FF0D4
:1047A200020E0101176F000E186FBDDC2CC017F14D
:1047B2002DC018F173DE290E0B6E960E0C6E7F0E55
:1047C2000D6E0D2EFED70C2EFCD70B2EFAD7020E35
:1047D200176F000E186FA7DC010E0101176F000E94
:1047E200186FA1DCEC0E01011D6F4C0E1E6F000E46
:1047F2001F6F63EC1FF0290E0B6E960E0C6E7F0E70
:104802000D6E0D2EFED70C2EFCD70B2EFAD73B6A5F
:104812003C6A020E0101176F000E186F84DC0E0E47
:1048220001011D6F4D0E1E6F000E1F6F63EC1FF016
:104832003BC017F13CC018F1800E0101196F000E48
:104842001A6FDDDDCB0E01011D6F010E1E6F13EC21
:104852001FF0800E0101176F000E186F1FDE3B4A1A
:104862003C2A150E0B6E4B0E0C6EBE0E0D6E0D2EEF
:10487200FED70C2EFCD70B2EFAD70000CAD7FFD7D3
:104D3A0010EE19F00B0E006E010E016E1F0EF66ECC
:0E4D4A004D0EF76E000EF86E05EC20F0120014
:10488200204469726563746F72793A20433A5C5FBF
:104892004D696B726F435C5F4D657350726F6A65F1
:1048A20074735F4D696B726F435C50494331384694
:1048B2005F455350383236365F5465737473200D3A
:0248C2000A00EA
:1048C4002054657374204C434420313630322032F6
:1048D40078313620656E2049324320766961205054
:1048E400434638373534206164646974696F6E6E89
:0748F400656C0D0A0D0A00BE
:1048FB000000007F000020820000488500007A88BD
:10490B0000401C8C0050438F0024749280961896A4
:10491B0020BC3E99286B6E9CF90215A0EC782DC13A
:04492B00CAF249E2A1
:10492F000000007FCDCC4C7B0AD723786F12037524
:10493F0017B75171ACC5276EBD37066B95BF56675C
:10494F0077CC2B645F700961FFE65B5D08E53C3C4B
:04495F006042221B75
:104963002055415254312076696120555342202D00
:104973003E20434F4D332031393230302C382C4ECA
:104983002C3120594154205465726D696E616C0D50
:024993000A0018
:1049950020536F75726365203A4553503832363669
:1049A5005F426173655F31384632364B32325F7430
:1049B500657374735F5F3139303831372E630D0A93
:0149C50000F1
:1049C6000100000008000000400000000002000096
:1049D600001000000080000000000400000020001D
:1049E6000000000100000008000000400000000078
:1049F60044657669636520617420616472657373CA
:104A060065202520336420736F6974202025303299
:104A16005820206973206E6F7420666F756E64006F
:104A260020536F7572636520455350383236365FB2
:104A3600426173655F31384632364B32325F746598
:104A46007374735F5F3139303831372E630D0A0066
:104A560020506F727420486172642055415254315F
:104A66002031393230302C4E2C382C31202852430C
:104A7600363D5458205243373D525829200D0A00DE
:104A860020434F4E464947203A2050313846323669
:104A96004B32325F464F53435F696E7465726E6583
:104AA6005F31364D687A2E6366677363680D0A0058
:104AB6002050726F6A6574203A204553503832365A
:104AC600365F426173655F31384632364B32325F4C
:0E4AD60074657374732E6D637070690D0A0041
:104AE400204861726477617265203A204361727470
:104AF4006520426173652031384632364B323220AC
:0E4B040020656E2032382050696E730D0A0055
:104B120044657669636520617420616472657373AC
:104B220065202520336420736F697420202530327C
:0E4B32005820090920666F756E64204F4B00F5
:104B4000010000000A00000064000000E80300000B
:104B500010270000A086010040420F0080969800B8
:084B600000E1F50500CA9A3BD3
:104B68002045637269742E207375722031657265F1
:104B7800206C69676E65206475204C4344203A2098
:014B8800002C
:104B89002045637269742E207375722032656D2019
:104B99006C69676E65206475204C4344203A200097
:104BA90001000000100000000001000000100000DA
:104BB90000000100000010000000000100000010CA
:104BC900204C43442032783136207375722050438B
:0B4BD90046383537342D31200D0A001E
:104BE40020496E697420446973706C6179204C4368
:0A4BF400442032783136203A2000C8
:104BFE0020496E697420554152543120313932307A
:0A4C0E00302C382C4E2C310D0A001A
:104C1800204C4344203278313620737572206275F7
:0A4C2800732049324331200D0A00C9
:104C320020416C696D2E203D20332E3020746F2070
:074C4200352E30560D0A006B
:104C490020464F534320696E7465726E6520313674
:064C59004D487A0D0A002F
:104C5F0020496E69742049324331203430304B681B
:044C6F007A0D0A00B0
:104C7300204D696B726F632050726F20372E353071
:034C83000D0A0017
:104C860048656C6C6F204920616D20616C697665A2
:014C9600001D
:104C9700202020202020202020202020202020200D
:014CA700000C
:104CA800303132333435363738394142434445465A
:014CB80000FB
:104CB9003031323334353637383961626364656689
:014CC90000EA
:104CCA007061756C666A756A6F20303132333435BB
:014CDA0000D9
:104CDB0048656C6C6F204920616D20616C6976654D
:014CEB0000C8
:104CEC007061756C666A756A6F2E667265652E6684
:014CFC0000B7
:104CFD0020202020202020202020202020202020A7
:014D0D0000A5
:104D0E00436F6D7074657572204A3D2020202020FF
:014D1E000094
:074D1F00286E756C6C290081
:044D26000000000089
:064D2A002020200D0A000C
:064D30002020200D0A0006
:044D3600200D0A0042
:020000040030CA
:0D000100281F3CFFBF81FF0FC00FE00F4024
:00000001FF
